:1000000000308A008F2A000000000A108A100A11AE
:10001000820763346F346D346D3461346E3464340C
:1000200020342034663475346E3463347434693467
:100030006F346E3400340A108A100A11820731348A
:1000400073346534743420344C344534443431349E
:1000500000340A108A100A118207323463346C3477
:10006000723420344C3445344434313400340A1072
:100070008A100A118207333473346534743420349F
:100080004C3445344434323400340A108A100A1196
:100090008207343463346C34723420344C34453445
:1000A0004434323400340A108A100A11820735347D
:1000B0006F346E3420344B34313400340A108A10DB
:1000C0000A11820736346F346634663420344B3478
:1000D000313400340A108A100A118207373472341E
:1000E000653461346434203473347734313400340B
:1000F0000A108A100A118207383472346534613468
:100100006434203473347734323400340A108A1063
:100110000A1182073F34683465346C34703400341B
:100120000A108A100A1182070A340D3463346F34BE
:100130006D346D3461346E3464342034253463346A
:1001400020346F346B3400340A108A100A1182078D
:100150002034523445344D344F34543445345B34B8
:10016000523453343234333432345D340A340A3442
:100170000D3400340A108A100A1182070A340D3433
:100180007334773431343D342534633400340A1009
:100190008A100A1182070A340D34733477343234EA
:1001A0003D3425346334003408308C00BE306600A2
:1001B000861ED8288F018C17EB288C13EB28031090
:1001C0008F0C861E8F170C17EB280C138C0BDF2857
:1001D0000F088D00F6281C308C1B07308D008D0B0E
:1001E000EF288C1BDD280C1BE528DF28AF2A083000
:1001F0008D00BE30660006178D170B298D13910CEC
:1002000003180613031C06170D170B290D138D0B6E
:10021000FF2806130B291E308400840B0D298D1B2B
:10022000FE280D1B062900348F010F0805208F0AB8
:100230009100F72011300F02031D15290D30910098
:10024000F7200A309100F72004308F002030910011
:10025000F7208F0B262931309100F72005308F00D1
:1002600020309100F7208F0B302901308F000F08CC
:100270001B208F0A9100F72009300F02031D372938
:100280000D309100F7200A309100F72004308F00E4
:1002900020309100F7208F0B482932309100F72051
:1002A00005308F0020309100F7208F0B522901304C
:1002B0008F000F0829208F0A9100F72009300F02C4
:1002C000031D59290D309100F7200A309100F720C5
:1002D00004308F0020309100F7208F0B6A293330D3
:1002E0009100F72005308F0020309100F7208F0B10
:1002F000742901308F000F0837208F0A9100F720F2
:1003000009300F02031D7B290D309100F7200A30C0
:100310009100F72004308F0020309100F7208F0BE0
:100320008C2934309100F72005308F002030910067
:10033000F7208F0B962901308F000F0845208F0A78
:100340009100F72009300F02031D9D290D30910007
:10035000F7200A309100F72004308F002030910000
:10036000F7208F0BAE2935309100F72006308F0033
:1003700020309100F7208F0BB82901308F000F0833
:1003800053208F0A9100F72006300F02031DBF296A
:100390000D309100F7200A309100F72004308F00D3
:1003A00020309100F7208F0BD02936309100F720B4
:1003B00005308F0020309100F7208F0BDA290130B3
:1003C0008F000F085E208F0A9100F72007300F0280
:1003D000031DE1290D309100F7200A309100F7202C
:1003E00004308F0020309100F7208F0BF229373036
:1003F0009100F72004308F0020309100F7208F0B00
:10040000FC2901308F000F086A208F0A9100F72025
:1004100009300F02031D032A0D309100F7200A3026
:100420009100F72004308F0020309100F7208F0BCF
:10043000142A38309100F72004308F0020309100CA
:10044000F7208F0B1E2A01308F000F0878208F0AAB
:100450009100F72009300F02031D252A0D3091006D
:10046000F7200A309100F72004308F0020309100EF
:10047000F7208F0B362A3F309100F72004308F0091
:1004800020309100F7208F0B402A01308F000F0899
:1004900086208F0A9100F72005300F02031D472A9E
:1004A0000D309100F7200A309100F720E82A07303C
:1004B0009100F7208F010F0890208F0A9100F720FC
:1004C0000A300F02031D5B2A0E089100F72020302E
:1004D0009100F7206F309100F7206B309100F720EA
:1004E0000034E030650005105722EA2AE03065004C
:1004F00005145722EC2AE030650085105722EE2AB9
:10050000E030650085145722F02ABE3066000614DC
:100510005722F22ABE30660006105722F42A8401C0
:100520008301BE30660006178C018C1D9F2A0730A0
:100530008101813084000008C0390F3880006400D8
:10054000813084000008C0390C048000E030650070
:10055000051465008514BE3066000610D4280D0809
:100560008E000E088C000D300C020319DC2A3F307F
:100570000C020319E72A31300C020319E92A323040
:100580000C020319EB2A33300C020319ED2A343024
:100590000C020319EF2A35300C020319F12A363008
:1005A0000C020319F32A37300C020319F52A3830EC
:1005B0000C0203190C2B232B8F010F08A4208F0A88
:1005C0009100F72011300F02031DDD2A232B14297F
:1005D000232B712A232B762A232B7B2A232B802A59
:1005E000232B852A232B8A2A232BBE30660000303A
:1005F000861801308C0030300C078F0090011008F5
:10060000BA20900A9100F72006301002031DFF2A3D
:100610000F089100F720232BBE306600003006192A
:1006200001308C0030300C078F0090011008C7207B
:10063000900A9100F72006301002031D162B0F08B8
:0A0640009100F720232BAE2A63007F
:00000001FF
